
 Start         Length     Name                   Class
 0001:00401000 00002934H .text                   CODE
 0002:00404000 000001F0H .itext                  ICODE
 0003:00405000 00000054H .data                   DATA
 0004:00406000 00000024H .bss                    BSS
 0005:00000000 00000000H .tls                    TLS


Detailed map of segments

 0001:00000000 0000014E C=CODE     S=.text    G=(none)   M=System   ACBP=A9
 0001:00000150 000001C3 C=CODE     S=.text    G=(none)   M=SysInit  ACBP=A9
 0001:00000314 0000001F C=CODE     S=.text    G=(none)   M=ccwizres ACBP=A9
 0001:00000334 00000006 C=CODE     S=.text    G=(none)   M=ImgList  ACBP=A9
 0001:0000033C 00000071 C=CODE     S=.text    G=(none)   M=Windows  ACBP=A9
 0001:000003B0 00000016 C=CODE     S=.text    G=(none)   M=Graphics ACBP=A9
 0001:000003C8 00000036 C=CODE     S=.text    G=(none)   M=Classes  ACBP=A9
 0001:00000400 00000006 C=CODE     S=.text    G=(none)   M=TypInfo  ACBP=A9
 0001:00000408 00000036 C=CODE     S=.text    G=(none)   M=SysUtils ACBP=A9
 0001:00000440 00000006 C=CODE     S=.text    G=(none)   M=Variants ACBP=A9
 0001:00000448 00000006 C=CODE     S=.text    G=(none)   M=VarUtils ACBP=A9
 0001:00000450 00000006 C=CODE     S=.text    G=(none)   M=Registry ACBP=A9
 0001:00000458 00000006 C=CODE     S=.text    G=(none)   M=IniFiles ACBP=A9
 0001:00000460 0000000E C=CODE     S=.text    G=(none)   M=IOUtils  ACBP=A9
 0001:00000470 00000006 C=CODE     S=.text    G=(none)   M=Themes   ACBP=A9
 0001:00000478 0000010E C=CODE     S=.text    G=(none)   M=Controls ACBP=A9
 0001:00000588 00000006 C=CODE     S=.text    G=(none)   M=SyncObjs ACBP=A9
 0001:00000590 00000006 C=CODE     S=.text    G=(none)   M=TimeSpan ACBP=A9
 0001:00000598 00000006 C=CODE     S=.text    G=(none)   M=ActnList ACBP=A9
 0001:000005A0 00000006 C=CODE     S=.text    G=(none)   M=Menus    ACBP=A9
 0001:000005A8 00000006 C=CODE     S=.text    G=(none)   M=UxTheme  ACBP=A9
 0001:000005B0 00000006 C=CODE     S=.text    G=(none)   M=MultiMon ACBP=A9
 0001:000005B8 0000013E C=CODE     S=.text    G=(none)   M=Forms    ACBP=A9
 0001:000006F8 00000006 C=CODE     S=.text    G=(none)   M=HelpIntfs ACBP=A9
 0001:00000700 00000006 C=CODE     S=.text    G=(none)   M=Dialogs  ACBP=A9
 0001:00000708 00000036 C=CODE     S=.text    G=(none)   M=ComCtrls ACBP=A9
 0001:00000740 00000006 C=CODE     S=.text    G=(none)   M=GraphUtil ACBP=A9
 0001:00000748 00000006 C=CODE     S=.text    G=(none)   M=ExtCtrls ACBP=A9
 0001:00000750 00000006 C=CODE     S=.text    G=(none)   M=Printers ACBP=A9
 0001:00000758 00000006 C=CODE     S=.text    G=(none)   M=Clipbrd  ACBP=A9
 0001:00000760 00000006 C=CODE     S=.text    G=(none)   M=FlatSB   ACBP=A9
 0001:00000768 00000006 C=CODE     S=.text    G=(none)   M=Buttons  ACBP=A9
 0001:00000770 00000036 C=CODE     S=.text    G=(none)   M=ccreg    ACBP=A9
 0001:000007A8 00000657 C=CODE     S=.text    G=(none)   M=ccwdlg   ACBP=A9
 0001:00000E00 0000000E C=CODE     S=.text    G=(none)   M=ToolsAPI ACBP=A9
 0001:00000E10 00000006 C=CODE     S=.text    G=(none)   M=XMLIntf  ACBP=A9
 0001:00000E18 00000006 C=CODE     S=.text    G=(none)   M=xmldom   ACBP=A9
 0001:00000E20 00000006 C=CODE     S=.text    G=(none)   M=msxmldom ACBP=A9
 0001:00000E28 00000006 C=CODE     S=.text    G=(none)   M=ComObj   ACBP=A9
 0001:00000E30 00000006 C=CODE     S=.text    G=(none)   M=DockForm ACBP=A9
 0001:00000E38 00000006 C=CODE     S=.text    G=(none)   M=IDEMessages ACBP=A9
 0001:00000E40 00000006 C=CODE     S=.text    G=(none)   M=DeskForm ACBP=A9
 0001:00000E48 00000006 C=CODE     S=.text    G=(none)   M=BaseDock ACBP=A9
 0001:00000E50 00000006 C=CODE     S=.text    G=(none)   M=PercentageDockTree ACBP=A9
 0001:00000E58 00000006 C=CODE     S=.text    G=(none)   M=CaptionedDockTree ACBP=A9
 0001:00000E60 00000006 C=CODE     S=.text    G=(none)   M=DockTabSet ACBP=A9
 0001:00000E68 00000006 C=CODE     S=.text    G=(none)   M=Tabs     ACBP=A9
 0001:00000E70 00000006 C=CODE     S=.text    G=(none)   M=DeskUtil ACBP=A9
 0001:00000E78 00000006 C=CODE     S=.text    G=(none)   M=TabDock  ACBP=A9
 0001:00000E80 00000006 C=CODE     S=.text    G=(none)   M=PlatformDefaultStyleActnCtrls ACBP=A9
 0001:00000E88 00000006 C=CODE     S=.text    G=(none)   M=ActnMan  ACBP=A9
 0001:00000E90 00000006 C=CODE     S=.text    G=(none)   M=ActnMenus ACBP=A9
 0001:00000E98 00000006 C=CODE     S=.text    G=(none)   M=ExtActns ACBP=A9
 0001:00000EA0 00000006 C=CODE     S=.text    G=(none)   M=ExtDlgs  ACBP=A9
 0001:00000EA8 00000006 C=CODE     S=.text    G=(none)   M=Mapi     ACBP=A9
 0001:00000EB0 00001637 C=CODE     S=.text    G=(none)   M=ccwiz    ACBP=A9
 0001:000024E8 0000044B C=CODE     S=.text    G=(none)   M=.ccpackD2010dsg ACBP=A9
 0002:00000000 00000006 C=ICODE    S=.itext   G=(none)   M=System   ACBP=A9
 0002:00000008 00000008 C=ICODE    S=.itext   G=(none)   M=ccwizres ACBP=A9
 0002:00000010 00000016 C=ICODE    S=.itext   G=(none)   M=Windows  ACBP=A9
 0002:00000028 00000006 C=ICODE    S=.itext   G=(none)   M=Graphics ACBP=A9
 0002:00000030 0000000E C=ICODE    S=.itext   G=(none)   M=Classes  ACBP=A9
 0002:00000040 00000006 C=ICODE    S=.itext   G=(none)   M=TypInfo  ACBP=A9
 0002:00000048 0000001E C=ICODE    S=.itext   G=(none)   M=SysUtils ACBP=A9
 0002:00000068 00000006 C=ICODE    S=.itext   G=(none)   M=Variants ACBP=A9
 0002:00000070 00000006 C=ICODE    S=.itext   G=(none)   M=VarUtils ACBP=A9
 0002:00000078 00000006 C=ICODE    S=.itext   G=(none)   M=Registry ACBP=A9
 0002:00000080 00000006 C=ICODE    S=.itext   G=(none)   M=IniFiles ACBP=A9
 0002:00000088 0000000E C=ICODE    S=.itext   G=(none)   M=IOUtils  ACBP=A9
 0002:00000098 00000006 C=ICODE    S=.itext   G=(none)   M=Themes   ACBP=A9
 0002:000000A0 00000006 C=ICODE    S=.itext   G=(none)   M=Controls ACBP=A9
 0002:000000A8 00000006 C=ICODE    S=.itext   G=(none)   M=SyncObjs ACBP=A9
 0002:000000B0 00000006 C=ICODE    S=.itext   G=(none)   M=TimeSpan ACBP=A9
 0002:000000B8 00000006 C=ICODE    S=.itext   G=(none)   M=ActnList ACBP=A9
 0002:000000C0 00000006 C=ICODE    S=.itext   G=(none)   M=Menus    ACBP=A9
 0002:000000C8 00000006 C=ICODE    S=.itext   G=(none)   M=UxTheme  ACBP=A9
 0002:000000D0 00000006 C=ICODE    S=.itext   G=(none)   M=MultiMon ACBP=A9
 0002:000000D8 00000006 C=ICODE    S=.itext   G=(none)   M=Forms    ACBP=A9
 0002:000000E0 00000006 C=ICODE    S=.itext   G=(none)   M=HelpIntfs ACBP=A9
 0002:000000E8 00000006 C=ICODE    S=.itext   G=(none)   M=Dialogs  ACBP=A9
 0002:000000F0 00000006 C=ICODE    S=.itext   G=(none)   M=ComCtrls ACBP=A9
 0002:000000F8 00000006 C=ICODE    S=.itext   G=(none)   M=GraphUtil ACBP=A9
 0002:00000100 00000006 C=ICODE    S=.itext   G=(none)   M=ExtCtrls ACBP=A9
 0002:00000108 00000006 C=ICODE    S=.itext   G=(none)   M=Printers ACBP=A9
 0002:00000110 00000006 C=ICODE    S=.itext   G=(none)   M=Clipbrd  ACBP=A9
 0002:00000118 00000006 C=ICODE    S=.itext   G=(none)   M=FlatSB   ACBP=A9
 0002:00000120 00000006 C=ICODE    S=.itext   G=(none)   M=Buttons  ACBP=A9
 0002:00000128 00000006 C=ICODE    S=.itext   G=(none)   M=ccreg    ACBP=A9
 0002:00000130 00000008 C=ICODE    S=.itext   G=(none)   M=ccwdlg   ACBP=A9
 0002:00000138 00000006 C=ICODE    S=.itext   G=(none)   M=ToolsAPI ACBP=A9
 0002:00000140 00000006 C=ICODE    S=.itext   G=(none)   M=XMLIntf  ACBP=A9
 0002:00000148 00000006 C=ICODE    S=.itext   G=(none)   M=xmldom   ACBP=A9
 0002:00000150 00000006 C=ICODE    S=.itext   G=(none)   M=msxmldom ACBP=A9
 0002:00000158 00000006 C=ICODE    S=.itext   G=(none)   M=ComObj   ACBP=A9
 0002:00000160 00000006 C=ICODE    S=.itext   G=(none)   M=DockForm ACBP=A9
 0002:00000168 00000006 C=ICODE    S=.itext   G=(none)   M=IDEMessages ACBP=A9
 0002:00000170 00000006 C=ICODE    S=.itext   G=(none)   M=DeskForm ACBP=A9
 0002:00000178 00000006 C=ICODE    S=.itext   G=(none)   M=BaseDock ACBP=A9
 0002:00000180 00000006 C=ICODE    S=.itext   G=(none)   M=PercentageDockTree ACBP=A9
 0002:00000188 00000006 C=ICODE    S=.itext   G=(none)   M=CaptionedDockTree ACBP=A9
 0002:00000190 00000006 C=ICODE    S=.itext   G=(none)   M=DockTabSet ACBP=A9
 0002:00000198 00000006 C=ICODE    S=.itext   G=(none)   M=Tabs     ACBP=A9
 0002:000001A0 00000006 C=ICODE    S=.itext   G=(none)   M=DeskUtil ACBP=A9
 0002:000001A8 00000006 C=ICODE    S=.itext   G=(none)   M=TabDock  ACBP=A9
 0002:000001B0 00000006 C=ICODE    S=.itext   G=(none)   M=PlatformDefaultStyleActnCtrls ACBP=A9
 0002:000001B8 00000006 C=ICODE    S=.itext   G=(none)   M=ActnMan  ACBP=A9
 0002:000001C0 00000006 C=ICODE    S=.itext   G=(none)   M=ActnMenus ACBP=A9
 0002:000001C8 00000006 C=ICODE    S=.itext   G=(none)   M=ExtActns ACBP=A9
 0002:000001D0 00000006 C=ICODE    S=.itext   G=(none)   M=ExtDlgs  ACBP=A9
 0002:000001D8 00000006 C=ICODE    S=.itext   G=(none)   M=Mapi     ACBP=A9
 0002:000001E0 00000008 C=ICODE    S=.itext   G=(none)   M=ccwiz    ACBP=A9
 0002:000001E8 00000005 C=ICODE    S=.itext   G=(none)   M=.ccpackD2010dsg ACBP=A9
 0003:00000000 00000030 C=DATA     S=.data    G=DGROUP   M=SysInit  ACBP=A9
 0003:00000030 0000000C C=DATA     S=.data    G=DGROUP   M=Windows  ACBP=A9
 0004:00000000 0000000C C=BSS      S=.bss     G=DGROUP   M=SysInit  ACBP=A9
 0004:0000000C 00000004 C=BSS      S=.bss     G=DGROUP   M=ccwizres ACBP=A9
 0004:00000010 00000008 C=BSS      S=.bss     G=DGROUP   M=Windows  ACBP=A9
 0004:00000018 00000008 C=BSS      S=.bss     G=DGROUP   M=ccwdlg   ACBP=A9
 0004:00000020 00000004 C=BSS      S=.bss     G=DGROUP   M=ccwiz    ACBP=A9


  Address             Publics by Name

 0002:000001E8       .ccpackD2010dsg..ccpackD2010dsg
 0001:00002914       .ccpackD2010dsg.@GetPackageInfoTable
 0001:0000291C       .ccpackD2010dsg.@PackageLoad
 0001:00002928       .ccpackD2010dsg.@PackageUnload
 0002:000000B8       ActnList.ActnList
 0001:00000598       ActnList.Finalization
 0002:000001B8       ActnMan.ActnMan
 0001:00000E88       ActnMan.Finalization
 0002:000001C0       ActnMenus.ActnMenus
 0001:00000E90       ActnMenus.Finalization
 0002:00000178       BaseDock.BaseDock
 0001:00000E48       BaseDock.Finalization
 0002:00000120       Buttons.Buttons
 0001:00000768       Buttons.Finalization
 0002:00000188       CaptionedDockTree.CaptionedDockTree
 0001:00000E58       CaptionedDockTree.Finalization
 0002:00000128       ccreg.ccreg
 0001:000007A0       ccreg.Finalization
 0001:00000780       ccreg.FindCustomContainerClass
 0001:00000778       ccreg.GetBaseContainer
 0001:00000790       ccreg.GetCustomContainerClass
 0001:00000798       ccreg.GetCustomContainerClassListCount
 0001:00000788       ccreg.GetCustomContainerUnit
 0001:00000770       ccreg.IsBaseContainer
 0004:0000001C       ccwdlg..2
 0001:000007A8       ccwdlg..TCCWDialog
 0004:00000018       ccwdlg.CCWDialog
 0002:00000130       ccwdlg.ccwdlg
 0001:00000DF8       ccwdlg.Finalization
 0001:00000CF0       ccwdlg.TCCWDialog.CCradioClick
 0001:00000CE8       ccwdlg.TCCWDialog.CCtreeChange
 0001:00000BE4       ccwdlg.TCCWDialog.GetContainerNode
 0001:00000DC8       ccwdlg.TCCWDialog.Loaded
 0001:00000CF8       ccwdlg.TCCWDialog.LoadNodes
 0001:00000C5C       ccwdlg.TCCWDialog.SelectImage
 0004:00000020       ccwiz..3
 0001:000013F8       ccwiz..TCCModuleCreator
 0001:00000FC4       ccwiz..TCCWizard
 0001:00001AA8       ccwiz..TOTAFile
 0002:000001E0       ccwiz.ccwiz
 0001:000024E0       ccwiz.Finalization
 0001:000019D4       ccwiz.Register
 0001:00001F10       ccwiz.TCCModuleCreator.Create
 0001:00002060       ccwiz.TCCModuleCreator.FormCreated
 0001:00002064       ccwiz.TCCModuleCreator.GetAncestorName
 0001:00002078       ccwiz.TCCModuleCreator.GetCreatorType
 0001:000020A4       ccwiz.TCCModuleCreator.GetExisting
 0001:000020A8       ccwiz.TCCModuleCreator.GetFileSystem
 0001:000020B8       ccwiz.TCCModuleCreator.GetFormName
 0001:0000211C       ccwiz.TCCModuleCreator.GetImplFileName
 0001:00002130       ccwiz.TCCModuleCreator.GetIntfFileName
 0001:00002140       ccwiz.TCCModuleCreator.GetMainForm
 0001:00002144       ccwiz.TCCModuleCreator.GetOwner
 0001:00002150       ccwiz.TCCModuleCreator.GetShowForm
 0001:00002154       ccwiz.TCCModuleCreator.GetShowSource
 0001:00002158       ccwiz.TCCModuleCreator.GetUnnamed
 0001:0000215C       ccwiz.TCCModuleCreator.NewFormFile
 0001:0000216C       ccwiz.TCCModuleCreator.NewImplSource
 0001:000024D0       ccwiz.TCCModuleCreator.NewIntfSource
 0001:00001C78       ccwiz.TCCWizard.AfterSave
 0001:00001C7C       ccwiz.TCCWizard.BeforeSave
 0001:00001C80       ccwiz.TCCWizard.Destroyed
 0001:00001D30       ccwiz.TCCWizard.Execute
 0001:00001E34       ccwiz.TCCWizard.GetAuthor
 0001:00001E70       ccwiz.TCCWizard.GetComment
 0001:00001EE8       ccwiz.TCCWizard.GetGlyph
 0001:00001C88       ccwiz.TCCWizard.GetIDString
 0001:00001CE0       ccwiz.TCCWizard.GetName
 0001:00001EC0       ccwiz.TCCWizard.GetPage
 0001:00001D24       ccwiz.TCCWizard.GetState
 0001:00001C84       ccwiz.TCCWizard.Modified
 0001:00001C08       ccwiz.TOTAFile.Create
 0001:00001C4C       ccwiz.TOTAFile.GetAge
 0001:00001C64       ccwiz.TOTAFile.GetSource
 0004:0000000C       ccwizres..1
 0002:00000008       ccwizres.ccwizres
 0001:0000032C       ccwizres.Finalization
 0002:00000038       Classes.Classes
 0001:000003F8       Classes.Finalization
 0001:000003E8       Classes.TComponent.SafeCallException
 0001:000003E0       Classes.TComponent.UpdateAction
 0001:000003F0       Classes.TComponent.UpdateRegistry
 0001:000003D8       Classes.TComponent.WriteState
 0001:000003C8       Classes.TPersistent.Assign
 0002:00000030       Classes.TThread.Create@
 0001:000003D0       Classes.TThread.Destroy@
 0002:00000110       Clipbrd.Clipbrd
 0001:00000758       Clipbrd.Finalization
 0002:000000F0       ComCtrls.ComCtrls
 0001:00000738       ComCtrls.Finalization
 0001:00000730       ComCtrls.TCustomTreeView.GetSelected
 0001:00000710       ComCtrls.TTreeNode.GetNext
 0001:00000708       ComCtrls.TTreeNode.SetSelected
 0001:00000718       ComCtrls.TTreeNodes.AddChildObject
 0001:00000720       ComCtrls.TTreeNodes.AddObject
 0001:00000728       ComCtrls.TTreeNodes.GetFirstNode
 0002:00000158       ComObj.ComObj
 0001:00000E28       ComObj.Finalization
 0002:000000A0       Controls.Controls
 0001:00000580       Controls.Finalization
 0001:000004C8       Controls.TControl.CreateTouchManager
 0001:00000488       Controls.TControl.GetAction
 0001:00000478       Controls.TControl.GetDragImages
 0001:00000480       Controls.TControl.GetEnabled
 0001:000004D0       Controls.TControl.GetFloatingDockSiteClass
 0001:000004B0       Controls.TControl.GetText
 0001:000004D8       Controls.TControl.InitiateAction
 0001:00000498       Controls.TControl.SetAutoSize
 0001:000004C0       Controls.TControl.SetBiDiMode
 0001:00000490       Controls.TControl.SetDragMode
 0001:000004A8       Controls.TControl.SetEnabled
 0001:000004A0       Controls.TControl.SetName
 0001:000004B8       Controls.TControl.SetText
 0001:00000558       Controls.TWinControl.AssignTo
 0001:00000560       Controls.TWinControl.CanAutoSize
 0001:00000548       Controls.TWinControl.CanResize
 0001:00000550       Controls.TWinControl.ConstrainedResize
 0001:000004E8       Controls.TWinControl.CreateHandle
 0001:000004F0       Controls.TWinControl.CustomAlignInsertBefore
 0001:000004F8       Controls.TWinControl.CustomAlignPosition
 0001:000004E0       Controls.TWinControl.DestroyWnd
 0001:00000570       Controls.TWinControl.DockReplaceDockClient
 0001:00000540       Controls.TWinControl.GetClientOrigin
 0001:00000538       Controls.TWinControl.GetControlExtents
 0001:00000518       Controls.TWinControl.GetDeviceContext
 0001:00000520       Controls.TWinControl.Invalidate
 0001:00000530       Controls.TWinControl.Repaint
 0001:00000508       Controls.TWinControl.SetBounds
 0001:00000568       Controls.TWinControl.SetParentBackground
 0001:00000500       Controls.TWinControl.SetParentDoubleBuffered
 0001:00000510       Controls.TWinControl.ShowControl
 0001:00000528       Controls.TWinControl.Update
 0001:00000578       Controls.TWinControl.UpdateControlOriginalParentSize
 0002:00000170       DeskForm.DeskForm
 0001:00000E40       DeskForm.Finalization
 0002:000001A0       DeskUtil.DeskUtil
 0001:00000E70       DeskUtil.Finalization
 0002:000000E8       Dialogs.Dialogs
 0001:00000700       Dialogs.Finalization
 0002:00000160       DockForm.DockForm
 0001:00000E30       DockForm.Finalization
 0002:00000190       DockTabSet.DockTabSet
 0001:00000E60       DockTabSet.Finalization
 0002:000001C8       ExtActns.ExtActns
 0001:00000E98       ExtActns.Finalization
 0002:00000100       ExtCtrls.ExtCtrls
 0001:00000748       ExtCtrls.Finalization
 0002:000001D0       ExtDlgs.ExtDlgs
 0001:00000EA0       ExtDlgs.Finalization
 0001:00000760       FlatSB.Finalization
 0002:00000118       FlatSB.FlatSB
 0001:000006F0       Forms.Finalization
 0002:000000D8       Forms.Forms
 0001:000005E8       Forms.TCustomForm.AfterConstruction
 0001:00000670       Forms.TCustomForm.AlignControls
 0001:000005F8       Forms.TCustomForm.BeforeDestruction
 0001:000006C0       Forms.TCustomForm.CloseQuery
 0001:000005E0       Forms.TCustomForm.Create
 0001:000005F0       Forms.TCustomForm.CreateNew
 0001:00000678       Forms.TCustomForm.CreateParams
 0001:00000688       Forms.TCustomForm.CreateWindowHandle
 0001:00000680       Forms.TCustomForm.CreateWnd
 0001:000006A0       Forms.TCustomForm.DefaultHandler
 0001:00000630       Forms.TCustomForm.DefineProperties
 0001:00000600       Forms.TCustomForm.Destroy
 0001:00000690       Forms.TCustomForm.DestroyHandle
 0001:00000698       Forms.TCustomForm.DestroyWindowHandle
 0001:00000608       Forms.TCustomForm.DoCreate
 0001:00000610       Forms.TCustomForm.DoDestroy
 0001:00000638       Forms.TCustomForm.GetClientRect
 0001:00000640       Forms.TCustomForm.GetFloating
 0001:00000618       Forms.TCustomForm.Loaded
 0001:00000620       Forms.TCustomForm.Notification
 0001:000006B0       Forms.TCustomForm.PaintWindow
 0001:000006E8       Forms.TCustomForm.QueryInterface
 0001:00000628       Forms.TCustomForm.ReadState
 0001:000006E0       Forms.TCustomForm.RequestAlign
 0001:000006B8       Forms.TCustomForm.Resizing
 0001:000006C8       Forms.TCustomForm.SetFocus
 0001:000006A8       Forms.TCustomForm.SetFocusedControl
 0001:00000658       Forms.TCustomForm.SetParent
 0001:00000648       Forms.TCustomForm.SetParentBiDiMode
 0001:000006D0       Forms.TCustomForm.ShowModal
 0001:000006D8       Forms.TCustomForm.UpdateActions
 0001:00000660       Forms.TCustomForm.ValidateRename
 0001:00000650       Forms.TCustomForm.WantChildKey
 0001:00000668       Forms.TCustomForm.WndProc
 0001:000005D8       Forms.TScrollingWinControl.AdjustClientRect
 0001:000005B8       Forms.TScrollingWinControl.AutoScrollEnabled
 0001:000005D0       Forms.TScrollingWinControl.AutoScrollInView
 0001:000005C0       Forms.TScrollingWinControl.DoGesture
 0001:000005C8       Forms.TScrollingWinControl.DoGetGestureOptions
 0001:000003C0       Graphics.Finalization
 0002:00000028       Graphics.Graphics
 0001:000003B8       Graphics.TBitmap.Create
 0001:000003B0       Graphics.TPicture.GetBitmap
 0001:00000740       GraphUtil.Finalization
 0002:000000F8       GraphUtil.GraphUtil
 0001:000006F8       HelpIntfs.Finalization
 0002:000000E0       HelpIntfs.HelpIntfs
 0001:00000E38       IDEMessages.Finalization
 0002:00000168       IDEMessages.IDEMessages
 0001:00000334       ImgList.TCustomImageList.GetBitmap
 0001:00000458       IniFiles.Finalization
 0002:00000080       IniFiles.IniFiles
 0001:00000468       IOUtils.Finalization
 0002:00000090       IOUtils.IOUtils
 0002:00000088       IOUtils.TPath.Create@
 0001:00000460       IOUtils.TPath.Destroy@
 0001:00000EA8       Mapi.Finalization
 0002:000001D8       Mapi.Mapi
 0001:000005A0       Menus.Finalization
 0002:000000C0       Menus.Menus
 0001:00000E20       msxmldom.Finalization
 0002:00000150       msxmldom.msxmldom
 0001:000005B0       MultiMon.Finalization
 0002:000000D0       MultiMon.MultiMon
 0001:00000E50       PercentageDockTree.Finalization
 0002:00000180       PercentageDockTree.PercentageDockTree
 0001:00000E80       PlatformDefaultStyleActnCtrls.Finalization
 0002:000001B0       PlatformDefaultStyleActnCtrls.PlatformDefaultStyleActnCtrls
 0001:00000750       Printers.Finalization
 0002:00000108       Printers.Printers
 0001:00000450       Registry.Finalization
 0002:00000078       Registry.Registry
 0001:00000588       SyncObjs.Finalization
 0002:000000A8       SyncObjs.SyncObjs
 0001:00000298       SysInit.@InitPkg
 0001:000002FC       SysInit.@PackageLoad
 0001:00000308       SysInit.@PackageUnload
 0001:00000188       SysInit.AllocTlsBuffer
 0001:00000244       SysInit.ExitProcessTLS
 0001:0000020C       SysInit.ExitThreadTLS
 0001:00000150       SysInit.FreeLibrary
 0001:00000194       SysInit.GetTlsSize
 0004:00000004       SysInit.HInstance
 0001:00000268       SysInit.InitializeModule
 0001:000001E0       SysInit.InitProcessTLS
 0001:0000019C       SysInit.InitThreadTLS
 0001:00000158       SysInit.LocalAlloc
 0001:00000160       SysInit.LocalFree
 0003:00000004       SysInit.Module
 0004:00000000       SysInit.ModuleIsLib
 0004:00000001       SysInit.ModuleIsPackage
 0001:00000168       SysInit.TlsAlloc
 0004:00000008       SysInit.tlsBuffer
 0001:00000170       SysInit.TlsFree
 0001:00000178       SysInit.TlsGetValue
 0003:00000000       SysInit.TlsIndex
 0005:00000000       SysInit.TlsLast
 0003:00000020       SysInit.TlsProc
 0001:00000180       SysInit.TlsSetValue
 0001:00000274       SysInit.UninitializeModule
 0001:00000070       System.@AfterConstruction
 0001:00000068       System.@ClassCreate
 0001:00000078       System.@HandleFinally
 0001:00000108       System.@IntfCast
 0001:000000F8       System.@IntfClear
 0001:00000100       System.@IntfCopy
 0001:00000080       System.@PackageLoad
 0001:00000088       System.@PackageUnload
 0001:00000090       System.@RunError
 0001:00000098       System.@UStrAddRef
 0001:000000A8       System.@UStrArrayClr
 0001:000000B0       System.@UStrAsg
 0001:000000C8       System.@UStrCat
 0001:000000D0       System.@UStrCat3
 0001:000000D8       System.@UStrCatN
 0001:000000A0       System.@UStrClr
 0001:000000E0       System.@UStrDelete
 0001:000000B8       System.@UStrLAsg
 0001:000000C0       System.@UStrLen
 0001:00000148       System.Finalization
 0001:00000140       System.LoadResString
 0001:000000E8       System.RegisterModule
 0002:00000000       System.System
 0001:00000110       System.TInterfacedObject.AfterConstruction
 0001:00000118       System.TInterfacedObject.BeforeDestruction
 0001:00000120       System.TInterfacedObject.NewInstance
 0001:00000128       System.TInterfacedObject.QueryInterface
 0001:00000130       System.TInterfacedObject._AddRef
 0001:00000138       System.TInterfacedObject._Release
 0001:00000000       System.TObject.ClassName
 0001:00000008       System.TObject.ClassParent
 0001:00000020       System.TObject.Create
 0001:00000058       System.TObject.DefaultHandler
 0001:00000028       System.TObject.Destroy
 0001:00000060       System.TObject.Dispatch
 0001:00000038       System.TObject.Equals
 0001:00000030       System.TObject.Free
 0001:00000018       System.TObject.FreeInstance
 0001:00000040       System.TObject.GetHashCode
 0001:00000010       System.TObject.NewInstance
 0001:00000048       System.TObject.SafeCallException
 0001:00000050       System.TObject.ToString
 0001:000000F0       System.UnregisterModule
 0001:00000408       SysUtils.AnsiCompareText
 0002:00000058       SysUtils.Exception.Create@
 0001:00000410       SysUtils.Exception.Destroy@
 0001:00000438       SysUtils.Finalization
 0001:00000420       SysUtils.FreeAndNil
 0001:00000418       SysUtils.StringReplace
 0002:00000060       SysUtils.SysUtils
 0002:00000050       SysUtils.TEncoding.Create@
 0001:00000430       SysUtils.TEncoding.Destroy@
 0002:00000048       SysUtils.TLanguages.Create@
 0001:00000428       SysUtils.TLanguages.Destroy@
 0001:00000E78       TabDock.Finalization
 0002:000001A8       TabDock.TabDock
 0001:00000E68       Tabs.Finalization
 0002:00000198       Tabs.Tabs
 0001:00000470       Themes.Finalization
 0002:00000098       Themes.Themes
 0002:000000B0       TimeSpan.TTimeSpan.Create@
 0001:00000590       TimeSpan.TTimeSpan.Destroy@
 0001:00000E08       ToolsAPI.Finalization
 0001:00000E00       ToolsAPI.RegisterPackageWizard
 0002:00000138       ToolsAPI.ToolsAPI
 0001:00000400       TypInfo.Finalization
 0002:00000040       TypInfo.TypInfo
 0001:000005A8       UxTheme.Finalization
 0002:000000C8       UxTheme.UxTheme
 0001:00000440       Variants.Finalization
 0002:00000068       Variants.Variants
 0001:00000448       VarUtils.Finalization
 0002:00000070       VarUtils.VarUtils
 0004:00000010       Windows..2
 0001:00000390       Windows.Finalization
 0001:0000033C       Windows.FreeLibrary
 0001:00000344       Windows.GetVersionEx
 0004:00000014       Windows.HtmlHelpModule
 0001:00000354       Windows.InitVersionInfo
 0001:0000034C       Windows.LoadIcon
 0003:00000030       Windows.Win32MajorVersion
 0003:00000034       Windows.Win32MinorVersion
 0003:00000038       Windows.Win32Platform
 0002:00000010       Windows.Windows
 0001:00000E18       xmldom.Finalization
 0002:00000148       xmldom.xmldom
 0001:00000E10       XMLIntf.Finalization
 0002:00000140       XMLIntf.XMLIntf


  Address             Publics by Value

 0001:00000000       System.TObject.ClassName
 0001:00000008       System.TObject.ClassParent
 0001:00000010       System.TObject.NewInstance
 0001:00000018       System.TObject.FreeInstance
 0001:00000020       System.TObject.Create
 0001:00000028       System.TObject.Destroy
 0001:00000030       System.TObject.Free
 0001:00000038       System.TObject.Equals
 0001:00000040       System.TObject.GetHashCode
 0001:00000048       System.TObject.SafeCallException
 0001:00000050       System.TObject.ToString
 0001:00000058       System.TObject.DefaultHandler
 0001:00000060       System.TObject.Dispatch
 0001:00000068       System.@ClassCreate
 0001:00000070       System.@AfterConstruction
 0001:00000078       System.@HandleFinally
 0001:00000080       System.@PackageLoad
 0001:00000088       System.@PackageUnload
 0001:00000090       System.@RunError
 0001:00000098       System.@UStrAddRef
 0001:000000A0       System.@UStrClr
 0001:000000A8       System.@UStrArrayClr
 0001:000000B0       System.@UStrAsg
 0001:000000B8       System.@UStrLAsg
 0001:000000C0       System.@UStrLen
 0001:000000C8       System.@UStrCat
 0001:000000D0       System.@UStrCat3
 0001:000000D8       System.@UStrCatN
 0001:000000E0       System.@UStrDelete
 0001:000000E8       System.RegisterModule
 0001:000000F0       System.UnregisterModule
 0001:000000F8       System.@IntfClear
 0001:00000100       System.@IntfCopy
 0001:00000108       System.@IntfCast
 0001:00000110       System.TInterfacedObject.AfterConstruction
 0001:00000118       System.TInterfacedObject.BeforeDestruction
 0001:00000120       System.TInterfacedObject.NewInstance
 0001:00000128       System.TInterfacedObject.QueryInterface
 0001:00000130       System.TInterfacedObject._AddRef
 0001:00000138       System.TInterfacedObject._Release
 0001:00000140       System.LoadResString
 0001:00000148       System.Finalization
 0001:00000150       SysInit.FreeLibrary
 0001:00000158       SysInit.LocalAlloc
 0001:00000160       SysInit.LocalFree
 0001:00000168       SysInit.TlsAlloc
 0001:00000170       SysInit.TlsFree
 0001:00000178       SysInit.TlsGetValue
 0001:00000180       SysInit.TlsSetValue
 0001:00000188       SysInit.AllocTlsBuffer
 0001:00000194       SysInit.GetTlsSize
 0001:0000019C       SysInit.InitThreadTLS
 0001:000001E0       SysInit.InitProcessTLS
 0001:0000020C       SysInit.ExitThreadTLS
 0001:00000244       SysInit.ExitProcessTLS
 0001:00000268       SysInit.InitializeModule
 0001:00000274       SysInit.UninitializeModule
 0001:00000298       SysInit.@InitPkg
 0001:000002FC       SysInit.@PackageLoad
 0001:00000308       SysInit.@PackageUnload
 0001:0000032C       ccwizres.Finalization
 0001:00000334       ImgList.TCustomImageList.GetBitmap
 0001:0000033C       Windows.FreeLibrary
 0001:00000344       Windows.GetVersionEx
 0001:0000034C       Windows.LoadIcon
 0001:00000354       Windows.InitVersionInfo
 0001:00000390       Windows.Finalization
 0001:000003B0       Graphics.TPicture.GetBitmap
 0001:000003B8       Graphics.TBitmap.Create
 0001:000003C0       Graphics.Finalization
 0001:000003C8       Classes.TPersistent.Assign
 0001:000003D0       Classes.TThread.Destroy@
 0001:000003D8       Classes.TComponent.WriteState
 0001:000003E0       Classes.TComponent.UpdateAction
 0001:000003E8       Classes.TComponent.SafeCallException
 0001:000003F0       Classes.TComponent.UpdateRegistry
 0001:000003F8       Classes.Finalization
 0001:00000400       TypInfo.Finalization
 0001:00000408       SysUtils.AnsiCompareText
 0001:00000410       SysUtils.Exception.Destroy@
 0001:00000418       SysUtils.StringReplace
 0001:00000420       SysUtils.FreeAndNil
 0001:00000428       SysUtils.TLanguages.Destroy@
 0001:00000430       SysUtils.TEncoding.Destroy@
 0001:00000438       SysUtils.Finalization
 0001:00000440       Variants.Finalization
 0001:00000448       VarUtils.Finalization
 0001:00000450       Registry.Finalization
 0001:00000458       IniFiles.Finalization
 0001:00000460       IOUtils.TPath.Destroy@
 0001:00000468       IOUtils.Finalization
 0001:00000470       Themes.Finalization
 0001:00000478       Controls.TControl.GetDragImages
 0001:00000480       Controls.TControl.GetEnabled
 0001:00000488       Controls.TControl.GetAction
 0001:00000490       Controls.TControl.SetDragMode
 0001:00000498       Controls.TControl.SetAutoSize
 0001:000004A0       Controls.TControl.SetName
 0001:000004A8       Controls.TControl.SetEnabled
 0001:000004B0       Controls.TControl.GetText
 0001:000004B8       Controls.TControl.SetText
 0001:000004C0       Controls.TControl.SetBiDiMode
 0001:000004C8       Controls.TControl.CreateTouchManager
 0001:000004D0       Controls.TControl.GetFloatingDockSiteClass
 0001:000004D8       Controls.TControl.InitiateAction
 0001:000004E0       Controls.TWinControl.DestroyWnd
 0001:000004E8       Controls.TWinControl.CreateHandle
 0001:000004F0       Controls.TWinControl.CustomAlignInsertBefore
 0001:000004F8       Controls.TWinControl.CustomAlignPosition
 0001:00000500       Controls.TWinControl.SetParentDoubleBuffered
 0001:00000508       Controls.TWinControl.SetBounds
 0001:00000510       Controls.TWinControl.ShowControl
 0001:00000518       Controls.TWinControl.GetDeviceContext
 0001:00000520       Controls.TWinControl.Invalidate
 0001:00000528       Controls.TWinControl.Update
 0001:00000530       Controls.TWinControl.Repaint
 0001:00000538       Controls.TWinControl.GetControlExtents
 0001:00000540       Controls.TWinControl.GetClientOrigin
 0001:00000548       Controls.TWinControl.CanResize
 0001:00000550       Controls.TWinControl.ConstrainedResize
 0001:00000558       Controls.TWinControl.AssignTo
 0001:00000560       Controls.TWinControl.CanAutoSize
 0001:00000568       Controls.TWinControl.SetParentBackground
 0001:00000570       Controls.TWinControl.DockReplaceDockClient
 0001:00000578       Controls.TWinControl.UpdateControlOriginalParentSize
 0001:00000580       Controls.Finalization
 0001:00000588       SyncObjs.Finalization
 0001:00000590       TimeSpan.TTimeSpan.Destroy@
 0001:00000598       ActnList.Finalization
 0001:000005A0       Menus.Finalization
 0001:000005A8       UxTheme.Finalization
 0001:000005B0       MultiMon.Finalization
 0001:000005B8       Forms.TScrollingWinControl.AutoScrollEnabled
 0001:000005C0       Forms.TScrollingWinControl.DoGesture
 0001:000005C8       Forms.TScrollingWinControl.DoGetGestureOptions
 0001:000005D0       Forms.TScrollingWinControl.AutoScrollInView
 0001:000005D8       Forms.TScrollingWinControl.AdjustClientRect
 0001:000005E0       Forms.TCustomForm.Create
 0001:000005E8       Forms.TCustomForm.AfterConstruction
 0001:000005F0       Forms.TCustomForm.CreateNew
 0001:000005F8       Forms.TCustomForm.BeforeDestruction
 0001:00000600       Forms.TCustomForm.Destroy
 0001:00000608       Forms.TCustomForm.DoCreate
 0001:00000610       Forms.TCustomForm.DoDestroy
 0001:00000618       Forms.TCustomForm.Loaded
 0001:00000620       Forms.TCustomForm.Notification
 0001:00000628       Forms.TCustomForm.ReadState
 0001:00000630       Forms.TCustomForm.DefineProperties
 0001:00000638       Forms.TCustomForm.GetClientRect
 0001:00000640       Forms.TCustomForm.GetFloating
 0001:00000648       Forms.TCustomForm.SetParentBiDiMode
 0001:00000650       Forms.TCustomForm.WantChildKey
 0001:00000658       Forms.TCustomForm.SetParent
 0001:00000660       Forms.TCustomForm.ValidateRename
 0001:00000668       Forms.TCustomForm.WndProc
 0001:00000670       Forms.TCustomForm.AlignControls
 0001:00000678       Forms.TCustomForm.CreateParams
 0001:00000680       Forms.TCustomForm.CreateWnd
 0001:00000688       Forms.TCustomForm.CreateWindowHandle
 0001:00000690       Forms.TCustomForm.DestroyHandle
 0001:00000698       Forms.TCustomForm.DestroyWindowHandle
 0001:000006A0       Forms.TCustomForm.DefaultHandler
 0001:000006A8       Forms.TCustomForm.SetFocusedControl
 0001:000006B0       Forms.TCustomForm.PaintWindow
 0001:000006B8       Forms.TCustomForm.Resizing
 0001:000006C0       Forms.TCustomForm.CloseQuery
 0001:000006C8       Forms.TCustomForm.SetFocus
 0001:000006D0       Forms.TCustomForm.ShowModal
 0001:000006D8       Forms.TCustomForm.UpdateActions
 0001:000006E0       Forms.TCustomForm.RequestAlign
 0001:000006E8       Forms.TCustomForm.QueryInterface
 0001:000006F0       Forms.Finalization
 0001:000006F8       HelpIntfs.Finalization
 0001:00000700       Dialogs.Finalization
 0001:00000708       ComCtrls.TTreeNode.SetSelected
 0001:00000710       ComCtrls.TTreeNode.GetNext
 0001:00000718       ComCtrls.TTreeNodes.AddChildObject
 0001:00000720       ComCtrls.TTreeNodes.AddObject
 0001:00000728       ComCtrls.TTreeNodes.GetFirstNode
 0001:00000730       ComCtrls.TCustomTreeView.GetSelected
 0001:00000738       ComCtrls.Finalization
 0001:00000740       GraphUtil.Finalization
 0001:00000748       ExtCtrls.Finalization
 0001:00000750       Printers.Finalization
 0001:00000758       Clipbrd.Finalization
 0001:00000760       FlatSB.Finalization
 0001:00000768       Buttons.Finalization
 0001:00000770       ccreg.IsBaseContainer
 0001:00000778       ccreg.GetBaseContainer
 0001:00000780       ccreg.FindCustomContainerClass
 0001:00000788       ccreg.GetCustomContainerUnit
 0001:00000790       ccreg.GetCustomContainerClass
 0001:00000798       ccreg.GetCustomContainerClassListCount
 0001:000007A0       ccreg.Finalization
 0001:000007A8       ccwdlg..TCCWDialog
 0001:00000BE4       ccwdlg.TCCWDialog.GetContainerNode
 0001:00000C5C       ccwdlg.TCCWDialog.SelectImage
 0001:00000CE8       ccwdlg.TCCWDialog.CCtreeChange
 0001:00000CF0       ccwdlg.TCCWDialog.CCradioClick
 0001:00000CF8       ccwdlg.TCCWDialog.LoadNodes
 0001:00000DC8       ccwdlg.TCCWDialog.Loaded
 0001:00000DF8       ccwdlg.Finalization
 0001:00000E00       ToolsAPI.RegisterPackageWizard
 0001:00000E08       ToolsAPI.Finalization
 0001:00000E10       XMLIntf.Finalization
 0001:00000E18       xmldom.Finalization
 0001:00000E20       msxmldom.Finalization
 0001:00000E28       ComObj.Finalization
 0001:00000E30       DockForm.Finalization
 0001:00000E38       IDEMessages.Finalization
 0001:00000E40       DeskForm.Finalization
 0001:00000E48       BaseDock.Finalization
 0001:00000E50       PercentageDockTree.Finalization
 0001:00000E58       CaptionedDockTree.Finalization
 0001:00000E60       DockTabSet.Finalization
 0001:00000E68       Tabs.Finalization
 0001:00000E70       DeskUtil.Finalization
 0001:00000E78       TabDock.Finalization
 0001:00000E80       PlatformDefaultStyleActnCtrls.Finalization
 0001:00000E88       ActnMan.Finalization
 0001:00000E90       ActnMenus.Finalization
 0001:00000E98       ExtActns.Finalization
 0001:00000EA0       ExtDlgs.Finalization
 0001:00000EA8       Mapi.Finalization
 0001:00000FC4       ccwiz..TCCWizard
 0001:000013F8       ccwiz..TCCModuleCreator
 0001:000019D4       ccwiz.Register
 0001:00001AA8       ccwiz..TOTAFile
 0001:00001C08       ccwiz.TOTAFile.Create
 0001:00001C4C       ccwiz.TOTAFile.GetAge
 0001:00001C64       ccwiz.TOTAFile.GetSource
 0001:00001C78       ccwiz.TCCWizard.AfterSave
 0001:00001C7C       ccwiz.TCCWizard.BeforeSave
 0001:00001C80       ccwiz.TCCWizard.Destroyed
 0001:00001C84       ccwiz.TCCWizard.Modified
 0001:00001C88       ccwiz.TCCWizard.GetIDString
 0001:00001CE0       ccwiz.TCCWizard.GetName
 0001:00001D24       ccwiz.TCCWizard.GetState
 0001:00001D30       ccwiz.TCCWizard.Execute
 0001:00001E34       ccwiz.TCCWizard.GetAuthor
 0001:00001E70       ccwiz.TCCWizard.GetComment
 0001:00001EC0       ccwiz.TCCWizard.GetPage
 0001:00001EE8       ccwiz.TCCWizard.GetGlyph
 0001:00001F10       ccwiz.TCCModuleCreator.Create
 0001:00002060       ccwiz.TCCModuleCreator.FormCreated
 0001:00002064       ccwiz.TCCModuleCreator.GetAncestorName
 0001:00002078       ccwiz.TCCModuleCreator.GetCreatorType
 0001:000020A4       ccwiz.TCCModuleCreator.GetExisting
 0001:000020A8       ccwiz.TCCModuleCreator.GetFileSystem
 0001:000020B8       ccwiz.TCCModuleCreator.GetFormName
 0001:0000211C       ccwiz.TCCModuleCreator.GetImplFileName
 0001:00002130       ccwiz.TCCModuleCreator.GetIntfFileName
 0001:00002140       ccwiz.TCCModuleCreator.GetMainForm
 0001:00002144       ccwiz.TCCModuleCreator.GetOwner
 0001:00002150       ccwiz.TCCModuleCreator.GetShowForm
 0001:00002154       ccwiz.TCCModuleCreator.GetShowSource
 0001:00002158       ccwiz.TCCModuleCreator.GetUnnamed
 0001:0000215C       ccwiz.TCCModuleCreator.NewFormFile
 0001:0000216C       ccwiz.TCCModuleCreator.NewImplSource
 0001:000024D0       ccwiz.TCCModuleCreator.NewIntfSource
 0001:000024E0       ccwiz.Finalization
 0001:00002914       .ccpackD2010dsg.@GetPackageInfoTable
 0001:0000291C       .ccpackD2010dsg.@PackageLoad
 0001:00002928       .ccpackD2010dsg.@PackageUnload
 0002:00000000       System.System
 0002:00000008       ccwizres.ccwizres
 0002:00000010       Windows.Windows
 0002:00000028       Graphics.Graphics
 0002:00000030       Classes.TThread.Create@
 0002:00000038       Classes.Classes
 0002:00000040       TypInfo.TypInfo
 0002:00000048       SysUtils.TLanguages.Create@
 0002:00000050       SysUtils.TEncoding.Create@
 0002:00000058       SysUtils.Exception.Create@
 0002:00000060       SysUtils.SysUtils
 0002:00000068       Variants.Variants
 0002:00000070       VarUtils.VarUtils
 0002:00000078       Registry.Registry
 0002:00000080       IniFiles.IniFiles
 0002:00000088       IOUtils.TPath.Create@
 0002:00000090       IOUtils.IOUtils
 0002:00000098       Themes.Themes
 0002:000000A0       Controls.Controls
 0002:000000A8       SyncObjs.SyncObjs
 0002:000000B0       TimeSpan.TTimeSpan.Create@
 0002:000000B8       ActnList.ActnList
 0002:000000C0       Menus.Menus
 0002:000000C8       UxTheme.UxTheme
 0002:000000D0       MultiMon.MultiMon
 0002:000000D8       Forms.Forms
 0002:000000E0       HelpIntfs.HelpIntfs
 0002:000000E8       Dialogs.Dialogs
 0002:000000F0       ComCtrls.ComCtrls
 0002:000000F8       GraphUtil.GraphUtil
 0002:00000100       ExtCtrls.ExtCtrls
 0002:00000108       Printers.Printers
 0002:00000110       Clipbrd.Clipbrd
 0002:00000118       FlatSB.FlatSB
 0002:00000120       Buttons.Buttons
 0002:00000128       ccreg.ccreg
 0002:00000130       ccwdlg.ccwdlg
 0002:00000138       ToolsAPI.ToolsAPI
 0002:00000140       XMLIntf.XMLIntf
 0002:00000148       xmldom.xmldom
 0002:00000150       msxmldom.msxmldom
 0002:00000158       ComObj.ComObj
 0002:00000160       DockForm.DockForm
 0002:00000168       IDEMessages.IDEMessages
 0002:00000170       DeskForm.DeskForm
 0002:00000178       BaseDock.BaseDock
 0002:00000180       PercentageDockTree.PercentageDockTree
 0002:00000188       CaptionedDockTree.CaptionedDockTree
 0002:00000190       DockTabSet.DockTabSet
 0002:00000198       Tabs.Tabs
 0002:000001A0       DeskUtil.DeskUtil
 0002:000001A8       TabDock.TabDock
 0002:000001B0       PlatformDefaultStyleActnCtrls.PlatformDefaultStyleActnCtrls
 0002:000001B8       ActnMan.ActnMan
 0002:000001C0       ActnMenus.ActnMenus
 0002:000001C8       ExtActns.ExtActns
 0002:000001D0       ExtDlgs.ExtDlgs
 0002:000001D8       Mapi.Mapi
 0002:000001E0       ccwiz.ccwiz
 0002:000001E8       .ccpackD2010dsg..ccpackD2010dsg
 0003:00000000       SysInit.TlsIndex
 0003:00000004       SysInit.Module
 0003:00000020       SysInit.TlsProc
 0003:00000030       Windows.Win32MajorVersion
 0003:00000034       Windows.Win32MinorVersion
 0003:00000038       Windows.Win32Platform
 0004:00000000       SysInit.ModuleIsLib
 0004:00000001       SysInit.ModuleIsPackage
 0004:00000004       SysInit.HInstance
 0004:00000008       SysInit.tlsBuffer
 0004:0000000C       ccwizres..1
 0004:00000010       Windows..2
 0004:00000014       Windows.HtmlHelpModule
 0004:00000018       ccwdlg.CCWDialog
 0004:0000001C       ccwdlg..2
 0004:00000020       ccwiz..3
 0005:00000000       SysInit.TlsLast


Line numbers for ccwizres(ccwizres.pas) segment .itext

   131 0002:00000008

Line numbers for ccwdlg(ccwdlg.pas) segment .text

    66 0001:00000BE4    67 0001:00000C04    68 0001:00000C17    70 0001:00000C1B
    71 0001:00000C2A    68 0001:00000C33    73 0001:00000C37    79 0001:00000C5C
    80 0001:00000C61    81 0001:00000C76    83 0001:00000C7B    84 0001:00000C89
    85 0001:00000CA2    86 0001:00000CC2    87 0001:00000CDA    88 0001:00000CE1
    92 0001:00000CE8    93 0001:00000CED    97 0001:00000CF0    98 0001:00000CF5
   104 0001:00000CF8   105 0001:00000D16   106 0001:00000D28   108 0001:00000D37
   109 0001:00000D40   110 0001:00000D4A   112 0001:00000D64   113 0001:00000D98
   106 0001:00000D99   114 0001:00000D9C   117 0001:00000DC8   118 0001:00000DCC
   119 0001:00000DD3   121 0001:00000DDF   122 0001:00000DE6   124 0001:00000DF4

Line numbers for ccwdlg(ccwdlg.pas) segment .itext

   126 0002:00000130

Line numbers for ccwiz(ccwiz.pas) segment .text

    91 0001:000019D4    92 0001:000019E7    93 0001:00001A11   108 0001:00001C08
   109 0001:00001C1D   110 0001:00001C26   111 0001:00001C30   114 0001:00001C4C
   115 0001:00001C4F   116 0001:00001C5C   119 0001:00001C64   120 0001:00001C6A
   121 0001:00001C74   126 0001:00001C78   130 0001:00001C7C   134 0001:00001C80
   138 0001:00001C84   141 0001:00001C88   142 0001:00001C8B   143 0001:00001C97
   146 0001:00001CE0   147 0001:00001CE3   148 0001:00001CEF   152 0001:00001D24
   153 0001:00001D2B   158 0001:00001D30   159 0001:00001D48   160 0001:00001D64
   161 0001:00001D72   163 0001:00001D84   164 0001:00001D99   167 0001:00001DDE
   169 0001:00001DF0   172 0001:00001E34   173 0001:00001E37   174 0001:00001E43
   177 0001:00001E70   178 0001:00001E73   179 0001:00001E7F   182 0001:00001EC0
   183 0001:00001EC3   184 0001:00001ECF   188 0001:00001EE8   189 0001:00001EF8
   196 0001:00001F10   197 0001:00001F4B   198 0001:00001F56   199 0001:00001F68
   200 0001:00001F73   201 0001:00001F9E   202 0001:00001FDB   203 0001:00001FFB
   208 0001:00002060   211 0001:00002064   212 0001:0000206A   213 0001:00002074
   216 0001:00002078   217 0001:0000207B   218 0001:00002087   222 0001:000020A4
   223 0001:000020A6   226 0001:000020A8   227 0001:000020AB   228 0001:000020B4
   233 0001:000020B8   234 0001:000020D1   235 0001:000020DC   236 0001:000020EE
   237 0001:000020F8   240 0001:0000211C   241 0001:00002122   242 0001:0000212C
   245 0001:00002130   246 0001:00002133   247 0001:0000213C   251 0001:00002140
   252 0001:00002142   255 0001:00002144   256 0001:00002147   257 0001:0000214E
   261 0001:00002150   262 0001:00002152   266 0001:00002154   267 0001:00002156
   271 0001:00002158   272 0001:0000215A   276 0001:0000215C   277 0001:0000215F
   278 0001:00002167   285 0001:0000216C   286 0001:00002191   287 0001:000021BB
   289 0001:000021CA   291 0001:000021D4   292 0001:000021FE   294 0001:0000223D
   296 0001:00002247   297 0001:0000225D   299 0001:0000226C   300 0001:00002298
   302 0001:000022A7   304 0001:000022B4   305 0001:000022DB   306 0001:00002302
   307 0001:00002329   308 0001:0000235A   310 0001:0000238B   311 0001:000023AB
   315 0001:000024D0   316 0001:000024D3   317 0001:000024DB

Line numbers for ccwiz(ccwiz.pas) segment .itext

   319 0002:000001E0

Line numbers for .ccpackD2010dsg(ccpackD2010dsg.dpk) segment .itext

    39 0002:000001E8

Bound resource files

ccwdlg.DFM
ccwiz.res
ccpackD2010dsg.res
ccpackD2010dsg.drf


Program entry point at 0002:000001E8
